:020000040000FA
:1000000085018316803081009501FC308500FF2337
:1000100090008312073099009F0199018E018F0192
:10002000900181018B01013085001030A000322049
:10003000A00B17284320A101272043205030A10006
:10004000272043205030A1002720322015280830D7
:10005000A000A10D031C2E2832202F284320A00B26
:10006000292808000B1D32280000E63081000B1102
:10007000013085000B1D3A280000E63081000B118D
:100080000230850008000B1D4328C83081000B1189
:10009000013085000B1D4A28C83081000B11023049
:0400A00085000800CF
:02400E00C43FAD
:104210004700E9006E00E9007200610074002E00A2
:1042200066007200650069006E006100670065004D
:10423000330030002F00310031002F0030003800F3
:00000001FF
